:040286001020804084
:1001950078087C007D007BFF7A0279867E007F04EB
:1001A5001200D3E4F50CF50D90E671E054EFF04341
:1001B500B410C2A4E054DFF043B420D2A5E0547FCC
:1001C500F043B480D2A7E054BFF043B440D2A605B3
:1001D5000DE50DAE0C7002050C14FF7C007D0412BC
:1001E50000F974082DF8E6F4F5A07F327E001202BE
:0301F5004880DC63
:10024800E4F50EF50FEF4E601EE4F50EF50F050F01
:10025800E50F7002050EE50FB420F3E50EB403EECA
:07026800EF1F70E11E80DEB4
:01026F00226C
:0801F8008F138E128D118C1083
:10020000E4F514F515E4FFFEFDFCAB13AA12A911E9
:10021000A810C312012F602FE4F514F5150515E59C
:100220001570020514E5156405451470F0E51324F6
:10023000FFF513E51234FFF512E51134FFF511E572
:070240001034FFF51080BE31
:010247002294
:0A027C0090E600E054E74410F02281
:0300000002027089
:0C027000787FE4F6D8FD75811502019539
:10000300E709F608DFFA8046E709F208DFFA803EDF
:1000130088828C83E709F0A3DFFA8032E309F608CC
:10002300DFFA8078E309F208DFFA807088828C8334
:10003300E309F0A3DFFA806489828A83E0A3F608E8
:10004300DFFA805889828A83E0A3F208DFFA804CC2
:1000530080D280FA80C680D4806980F28033801099
:1000630080A680EA809A80A880DA80E280CA803302
:1000730089828A83ECFAE493A3C8C582C8CCC5837A
:10008300CCF0A3C8C582C8CCC583CCDFE9DEE7804A
:100093000D89828A83E493A3F608DFF9ECFAA9F0C9
:1000A300EDFB2289828A83ECFAE0A3C8C582C8CC1F
:1000B300C583CCF0A3C8C582C8CCC583CCDFEADE38
:1000C300E880DB89828A83E493A3F208DFF980CC9A
:1000D30088F0EF60010E4E60C388F0ED2402B40493
:1000E3000050B9F582EB2402B4040050AF2323453A
:0600F3008223900053730C
:1000F900C2D5EC30E709B2D5E4C39DFDE49CFCEE22
:1001090030E715B2D5E4C39FFFE49EFE120140C358
:10011900E49DFDE49CFC800312014030D507C3E453
:060129009FFFE49EFE2290
:10012F00EB9FF5F0EA9E42F0E99D42F0E89C45F026
:01013F00229D
:10014000BC000BBE0029EF8DF084FFADF022E4CCA3
:10015000F875F008EF2FFFEE33FEEC33FCEE9DEC6C
:10016000984005FCEE9DFE0FD5F0E9E4CEFD22EDB2
:10017000F8F5F0EE8420D21CFEADF075F008EF2FFC
:10018000FFED33FD4007985006D5F0F222C398FDED
:050190000FD5F0EA228A
:00000001FF
